:020000040000FA
:06000000D1EF03F0120035
:0600080004EF04F01200F9
:060018000CEF04F01200E1
:06002A000100CE070000FA
:080030006A000000020000005C
:08003800126A1E0E716E040134
:10004000400E096F200E0A6F040E0B6F880E086FAA
:100050000401200E0E6F040E0F6F400E0C6F120085
:10006000550EA76EAA0EA76EA68212000401140EEA
:10007000226F010E236F1200106A04012151105CDF
:100080001CE2166A176A22511024F36E23511620BF
:10009000F46E24511720F86EF4CFF7FFF3CFF6FF7C
:1000A0000800F550116E1050EA6A250FE96E040E33
:1000B000EA2211C0EFFF102AE0D7F86A1200F00E12
:1000C00004012217840EA66E106A04012151105CEF
:1000D00023E21050EA6A250FE96E040EEA22EFCF00
:1000E00018F01050156E166A176A22511024F36E1C
:1000F00023511620F46E24511720F86EF4CFF7FF29
:10010000F3CFF6FF18C0F5FF0C000F0E10140F0808
:1001100001E1A6DF102AD9D71200940EA66E106A4C
:1001200004012151105C1DE21050156E166A060E76
:10013000D89015361636E804FBE1176A16BE176824
:10014000040122511524F36E23511620F46E24511C
:100150001720F86EF4CFF7FFF3CFF6FF81DF102AF8
:10016000DFD7F86A1200A66A106A04012151105CF8
:100170000EE222511024A96EA6801050EA6A250FC3
:10018000E96E040EEA22A8CFEFFF102AEED7120084
:10019000106A04012151105C12E222511024A96E50
:1001A0001050EA6A250FE96E040EEA22EF50A86E9D
:1001B000040EA66E55DFA6B2FED7102AEAD71200AB
:1001C000C40EA66E106A04012151105C1FE210508B
:1001D000EA6A250FE96E040EEA22EFCF18F01050FC
:1001E000156E166A176A22511024F36E23511620D9
:1001F000F46E24511720F86EF4CFF7FFF3CFF6FF1B
:1002000018C0F5FF0C002CDF102ADDD7F86A1200A9
:1002100079D8060E015C03E36D50020B01E071D04A
:10022000120410E104010CBF0CD00401400E096F50
:10023000400E040108170401087D880E040108130C
:10024000126A5FD0040108BF5CD0106A040120511B
:10025000320A3BE0CD0A2DE0F80A27E0020A21E04D
:10026000010A1BE0070A15E0010A0FE0030A09E092
:10027000070A07E0060A01E035D0F8DE040E106E2A
:1002800032D0FADE050E10262ED019DF010E106EC8
:100290002AD043DF010E106E26D065DF050E102632
:1002A00022D076DF010E106E1ED08ADF010E106E96
:1002B0001AD06D96136A146A1306000E145A13505E
:1002C000141001E0F9D7FF000ED0030E0401215DE8
:1002D00002E1010E106E040E0401215D02E1010E27
:1002E000106E01D000D0010E126E10500AE010C046
:1002F0000DF4400E04010C1704010C7D880E04015E
:100300000C13120000016A516B1104E1200E6A6F98
:100310004E0E6B6F6A07000E6B5B6DA208D06A51C0
:100320006B112DE18B708B50010B12E125D0015028
:1003300002E18B9021D0010402E18B8009D0020EF2
:10034000015C02E18B8018D0030E015C03E18B900D
:100350008B821200050E015C05E16A516B110FE101
:100360008B700AD0060E015C0AE16A516B1107E13D
:100370008B708B50010B02E08B9212008B8212006B
:100380006C500BE1040100513C0BE842E8420D08BF
:1003900002E1D2EF01F0DAEF01F0040E6C5C01E152
:1003A00017D81200056A066A0B6A0C6AFBEC02F0A9
:1003B00058EF02F0020E055C09E157D8040100BDB8
:1003C00002D0C80E01D0880E006F120096EF02F026
:1003D000040E015C09E112C46EFF6E50000802E2D7
:1003E000050E01D0030E016E050409E10AD80401CF
:1003F00004BD02D0C80E01D0880E046F120096EF23
:1004000002F0080E0B5C000E0C5802E20B5001D0FB
:10041000080E0E6EE8CF05F4166AE8500B5E165013
:100420000C5A180E096E040E0A6E0E501DE002A240
:1004300007D007C0F6FF08C0F7FF0800F55005D049
:1004400007C0E9FF08C0EAFFEF50E66E09C0E9FF08
:100450000AC0EAFFE552E750EF6E072A000E0822B5
:10046000092A0A220E06E1D7120001C40FF00F502C
:100470000B240B6E000E0C200C6E180E076E040E73
:10048000086E0F5014E007C0E9FF08C0EAFFEF5004
:10049000E66E09C0E9FF0AC0EAFFE552E750EF6ED9
:1004A000092A000E0A22072A08220F06EAD712009C
:1004B0006D9806500BE10401080E016F100E026FDB
:1004C000040E036F840E006F04011ED0040110AFF0
:1004D0001DD00B50165D0C50175904E216C40BF0DA
:1004E00017C40CF08EDF010E056E0401080E016FBB
:1004F000100E026F040E036F800E006F0401180EC1
:10050000066F040E076FC80E046F1200020E056E10
:100510000401056BC80E046F0401080E016F180E6C
:10052000026F040E036FC80E006F1200056A04010B
:10053000080E016F100E026F040E036F8C0E006F19
:060540000401046B12002F
:0A054600080E6D6E6DBAFED7686AEC
:10055000110E696E020E016E12006850040B09E064
:100560006950040B06E06D92699468A402D0689407
:10057000FCD76850010B04E06950010B01E024D85E
:100580006850100B0AE06950100B07E06984689806
:100590006D82A19AA08A0300A19A6850200B06E000
:1005A0006950200B03E070B07090689A030E015CF4
:1005B00001E209D06850080B06E06950080B03E01F
:1005C000C0EC01F068961200686A7B0E696E6E6A74
:1005D000160E706E68A608D0689600000000000035
:1005E000000000000000F6D76D9896EC02F0036A58
:0605F000030E016E120073
:0A05F60004011051600BE842E842D6
:10060000E842E842E842000901E012001151080AFC
:100610002FE0010A2BE00F0A08E0030A01E01200B4
:10062000010E066E040E016E1200010E066E130519
:1006300006E13E0E076E070E086E120E11D0020E76
:10064000135D06E1500E076E070E086E200E08D0EF
:10065000030E135D08E1700E076E070E086E040EA0
:100660000B6E0C6A01D0066A0282120042EF03F0A0
:10067000010E066E030E076E000E086E0292010E4A
:100680000B6E1200010E066E12C403F0040112512B
:1006900003E1050E016E1200060E016E1CEF00F064
:1006A0002A0EF66E000EF76E000EF86E00010900BD
:1006B000F550656F0900F550666F03E1656701D07D
:1006C0003DD00900F550606F0900F550616F0900D9
:1006D000F550626F09000900F550E96E0900F55008
:1006E000EA6E090009000900F550636F0900F55032
:1006F000646F09000900F6CF67F0F7CF68F0F8CF14
:1007000069F060C0F6FF61C0F7FF62C0F8FF00014A
:10071000635302E1645307E00900F550EE6E63078E
:10072000F8E26407F9D767C0F6FF68C0F7FF69C051
:0E073000F8FF00016507000E665BBFD71200E0
:02073E001201A6
:10074000000200000008D8040B00010000000001B6
:1007500009022000010100803209040000020000AB
:10076000000007050102400000070581024000006B
:040770000403090471
:0C077400C150006E0F0EC11282A404D010
:100780000050C16E00EF04F08B6AFC0E946E140EE4
:100790006F6EA3EC02F0ADEC02F008EC01F0FBD7B9
:0207A000120045
:0E07A20013EE00F023EE00F0F86A1A9C50EC03
:0E07B00003F0E6EC03F0BAEC03F0FBD7120006
:0207BE0000EE4B
:0C07C00000F00F0EEE6AEA62FDD7120096
:0207CC00120019
:0207CE00000029
:020000040030CA
:0100000024DB
:010001000EF0
:010002003AC3
:010003001EDE
:010005008179
:010006008178
:010008000FE8
:010009008076
:01000A000FE6
:01000B00A054
:01000C000FE4
:01000D0040B2
:00000001FF
